:100000000C94D6060C941D070C941D070C941D0728
:100010000C941D070C941D070C941D070C941D07D0
:100020000C941D070C941D070C9432160C940417A5
:100030000C94DB250C941D070C941D070C941D07D4
:100040000C941D070C941D070C941D070C941D07A0
:100050000C941D070C947B260C941D070C941D0713
:100060000C941D070C9479090C941D070C941D0722
:100070000C941D070C941D070C941D070C941D0770
:100080000C941D070C941D070C941D070C941D0760
:100090000C941D070C941D070C941D070C941D0750
:1000A0000C941D070C941D070C941D07B70EBB0E76
:1000B000BF0EC30EC70ECB0ECF0ED30ED70EDB0E68
:1000C000DF0EE30EE70EEB0EEF0EF30EF70EFB0E58
:1000D000FF0E030F070F0B0F0F0F130F170F1B0F41
:1000E0001F0F230F270F2B0F2F0F330F370F3B0F30
:1000F0003F0F430F830FB50E470F490F4B0F4D0FA7
:10010000510F550F590F5D0F620F670F6B0F6F0F78
:10011000730F770F7B0F810F810F810F810F810F7D
:10012000810F810F810F810F810F810F810F810F4F
:10013000810F810F810F810F810F810F7F0F711749
:100140009317811893178118D817FB178118501827
:100150006318631B631B921B921BF01B2E1C481E13
:10016000481E471C481E481D481D1C1E481E481E90
:10017000331E8080352B787939808080210877067E
:1001800007808080201A7A1B168080801E8029803C
:10019000808080808080808080808080221580198F
:1001A000098080801F147B1D0480808023172C050C
:1001B0000A808080260C00360E80808025187610FC
:1001C0000D808080241C80110B80808027127E3758
:1001D0000F8080802A804F7D28808080743051522B
:1001E000328080802D137C38338080802E2F507594
:1001F000348025630025730D0A00522C310D0A004E
:1002000053592C464646340D0A0053482C3030339F
:10021000430D0A00537E2C360D0A0053572C3830FC
:1002200030300D0A00534D2C340D0A0053532C4B23
:100230006579626F6172642F4D6F7573650D0A0089
:10024000532D2C546D6B42540D0A0053462C310D26
:100250000A002D2D2D0D0A0045786974696E6720FE
:10026000636F6E666967206D6F6465202E2E2E0A9F
:10027000002B0D0A00760D0A0024242400456E741C
:100280006572696E6720636F6E666967206D6F6463
:1002900065202E2E2E0A00522C310D0A0053522CAE
:1002A0005A0D0A00555342206D6F64650A0041756E
:1002B000746F206D6F64650A00253032750A002561
:1002C0003032753A00253032753A004241543A20B6
:1002D00025756D560900757074696D653A20253075
:1002E000327520253032753A253032753A25303254
:1002F000750A00564255533A2025580A0052656D3A
:100300006F746557616B657570456E61626C65648D
:100310003A2025580A000A003F004C4F5700444934
:10032000534348470043484152470046554C4C0010
:10033000626174746572793A200055534220537497
:100340006174653A2025730A00636F6E6669675FA2
:100350006D6F64653A2025580A00726E34325F6111
:1003600075746F636F6E6E656374696E6728293A82
:100370002025580A00726E34323A2025730A00662E
:100380006F7263655F7573623A2025580A00707258
:100390006F746F636F6C3A2025730A000A2D2D2D40
:1003A0002D2D20524E2D343220696E666F202D2D5A
:1003B0002D2D2D0A00753A20202020202020746F3A
:1003C00067676C6520466F72636520555342206DE8
:1003D0006F64650A00703A20202020202020706180
:1003E0006972696E670A00536C636B3A20202020A3
:1003F000524E2D343220696E697469616C697A6578
:100400000A0044656C3A2020202020656E746572D5
:100410002F6578697420524E2D343220636F6E66DA
:100420006967206D6F64650A00623A2020202020F1
:1004300020206261747465727920766F6C746167D4
:10044000650A00693A20202020202020524E2D34B9
:100450003220696E666F0A000A0A2D2D2D2D2D207F
:10046000426C7565746F6F746820524E2D34322063
:1004700048656C70202D2D2D2D2D0A0025303275EC
:100480003A253032753A253032750925756D560A90
:10049000004C4544207374617475733A20253032E2
:1004A000580A002025303258002563005B735D0038
:1004B0004B6579626F6172642073746172740A00B3
:1004C000524E2D343220696E69740A000A55534227
:1004D00020696E69740A005B445D005B435D001235
:1004E00003480048004B00420020006D006F00648C
:1004F0000000000E0374002E006D002E006B002E15
:100500000000000403090409028D00050100A03267
:100510000904000001030101000921110100012269
:1005200040000705810308000A09040100010301D6
:100530000200092111010001224D00070582030874
:10054000000A090402000103000000092111010052
:10055000012236000705830308000A09040300028C
:100560000300000009211101000122220007058477
:100570000320000107050403200001090404000111
:10058000030000000921110100012239000705853F
:10059000032000011201100100000008EDFE42429C
:1005A00004010102000105010906A101050719E086
:1005B00029E7150025019508750181020508190133
:1005C00029059505750191029501750391010507AE
:1005D000190029F71500250195F875018102C0065B
:1005E00031FF0974A1010975150026FF00952075DA
:1005F0000881020976150026FF00952075089102F2
:10060000C005010980A101850216810026B7001AE4
:1006100081002AB700751095018100C0050C090101
:10062000A1018503160100269C021A01002A9C02E2
:10063000751095018100C005010902A1010901A100
:100640000005091901290515002501950575018188
:1006500002950175038101050109300931158125D4
:100660007F95027508810609381581257F950175EA
:10067000088106050C0A38021581257F9501750849
:100680008106C0C005010906A101050719E029E797
:1006900015002501950875018102950175088101F4
:1006A0000508190129059505750191029501750344
:1006B00091010507190029FF150026FF0095067511
:1006C000088100C0636F6E73756D65723A202530C6
:1006D00034580A0073797374656D3A2025303458A4
:1006E0000A000A002530325820006B6579626F617C
:1006F00072643A20004C45443A20253032580A00B2
:10070000253032583A202530386225730A00722F7E
:10071000632030313233343536370A0064656C5F1C
:100720006B65795F6269743A2063616E2774206437
:10073000656C3A20253032580A006164645F6B654D
:10074000795F6269743A2063616E27742061646422
:100750003A20253032580A004F6E6573686F743A3C
:100760002074696D656F75740A00290A002575008B
:100770002F002575005D28002564002000256400F9
:10078000200025640020002564007C0025303258BC
:10079000006D6F7573656B6579205B62746E7C7834
:1007A0002079207620685D287265702F61636C293E
:1007B0003A205B006D6B5F776865656C5F74696D8F
:1007C000655F746F5F6D6178203D2025640A006D60
:1007D0006B5F776865656C5F6D61785F7370656589
:1007E00064203D2025640A006D6B5F74696D655F50
:1007F000746F5F6D6178203D2025640A006D6B5F2A
:100800006D61785F7370656564203D2025640A0022
:100810006D6B5F696E74657276616C203D20256436
:100820000A006D6B5F64656C6179203D2025640A68
:10083000006D6B5F776865656C5F74696D655F748B
:100840006F5F6D6178203D2025640A006D6B5F77D6
:100850006865656C5F6D61785F7370656564203D88
:100860002025640A006D6B5F74696D655F746F5F4E
:100870006D6178203D2025640A006D6B5F6D6178A5
:100880005F7370656564203D2025640A006D6B5FB1
:10089000696E74657276616C203D2025640A006D76
:1008A0006B5F64656C6179203D2025640A000A0055
:1008B000257500363A20776865656C5F74696D65EB
:1008C0005F746F5F6D61783A20000A00257500350E
:1008D0003A20776865656C5F6D61785F73706565F8
:1008E000643A20000A00257500343A2074696D6569
:1008F0005F746F5F6D61783A20000A0025750033E0
:100900003A206D61785F73706565643A20000A0073
:10091000257500323A20696E74657276616C286DB7
:1009200073293A20000A00257500313A2064656C6D
:100930006179282A31306D73293A20000A092D2067
:1009400056616C756573202D0A004D3E004D25647F
:100950003E20003F007365742064656661756C74A9
:100960000A00433E200077686572652064656C74F8
:10097000613A20637572736F723D25642C2077682D
:1009800065656C3D25640A53656520687474703A2A
:100990002F2F656E2E77696B6970656469612E6FA4
:1009A00072672F77696B692F4D6F7573655F6B6524
:1009B00079730A000A092D204D6F7573656B65798F
:1009C000202D0A4553432F713A09717569740A3114
:1009D0003A0964656C6179282A31306D73290A32CD
:1009E0003A09696E74657276616C286D73290A33F1
:1009F0003A096D61785F73706565640A343A097409
:100A0000696D655F746F5F6D61780A353A09776863
:100A100065656C5F6D61785F73706565640A363A11
:100A200009776865656C5F74696D655F746F5F6D8C
:100A300061780A0A703A097072696E742076616C86
:100A40007565730A643A0973657420646566617537
:100A50006C74730A75703A092B310A646F776E3AB9
:100A6000092D310A706775703A092B31300A7067A9
:100A7000646F776E3A092D31300A0A7370656564C8
:100A8000203D2064656C7461202A206D61785F735D
:100A900070656564202A2028726570656174202F56
:100AA0002074696D655F746F5F6D6178290A003F1E
:100AB000004D3E2000433E20004C25640A000A09F8
:100AC0002D20436F6E736F6C65202D0A4553432FA5
:100AD000713A09717569740A6D3A096D6F757365BC
:100AE0006B65790A000A092D204D61676963202D25
:100AF0000A643A0964656275670A783A096465624E
:100B00007567206D61747269780A6B3A0964656271
:100B10007567206B6579626F6172640A6D3A09646A
:100B200065627567206D6F7573650A763A0976653B
:100B30007273696F6E0A733A097374617475730A1C
:100B4000633A09636F6E736F6C65206D6F64650A3D
:100B5000302D343A096C61796572302D3428463174
:100B6000302D4634290A506175733A09626F6F74EB
:100B70006C6F616465720A6E3A094E4B524F0A00FF
:100B80003F004E4B524F3A206F66660A004E4B5262
:100B90004F3A206F6E0A0074696D65725F7265610D
:100BA00064333228293A202530346C580A006B65AA
:100BB00079626F6172645F6E6B726F3A2025580ABA
:100BC000006B6579626F6172645F69646C653A207D
:100BD00025580A006B6579626F6172645F70726F8D
:100BE000746F636F6C3A2025580A00686F73745FE6
:100BF0006B6579626F6172645F6C65647328293A12
:100C00002025580A000A092D205374617475732039
:100C10002D0A004743433A20342E392E32204156C4
:100C2000522D4C4942433A20312E382E3073766E85
:100C3000204156525F415243483A20617672350A4C
:100C4000004F5054494F4E533A204C554641204D89
:100C50004F5553454B45592045585452414B4559E2
:100C600020434F4E534F4C4520434F4D4D414E4432
:100C7000204E4B524F204B45594D41505F534543F9
:100C800054494F4E20343039360A004255494C44BD
:100C90003A20316237366561342D64697274792087
:100CA0002831383A30373A3233204D6172203136AC
:100CB0002032303138290A005649443A20307846EB
:100CC00045454428742E6D2E6B2E29205049443AF8
:100CD000203078343234322848484B42206D6F64DB
:100CE00029205645523A203078303130340A0044B9
:100CF0004553433A20742E6D2E6B2E206B6579621E
:100D00006F617264206669726D7761726520666FCB
:100D1000722048484B42206D6F640A000A092D205A
:100D200056657273696F6E202D0A000A6D6F7573B8
:100D3000653A206F66660A000A6D6F7573653A2022
:100D40006F6E0A000A6B6579626F6172643A206F98
:100D500066660A000A6B6579626F6172643A206F99
:100D60006E0A000A6D61747269783A206F66660ACD
:100D7000000A6D61747269783A206F6E0A000A6425
:100D8000656275673A206F6E0A000A64656275676E
:100D90003A206F66660A000A0A626F6F746C6F61B0
:100DA0006465722E2E2E2000433E200011241FBEAB
:100DB000CFEFDAE0DEBFCDBF04B603FE27C08091DF
:100DC0002E0490912F04A0913004B091310487300B
:100DD000904BA740B04BD1F410922E0410922F04E8
:100DE000109230041092310414BE84B7877F84BF00
:100DF0000FB6F894A8958091600088618093600098
:100E0000109260000FBEE0E0F8E3099511E0A0E069
:100E1000B1E0E8E4FEE502C005900D92A03AB1070A
:100E2000D9F724E0A0EAB1E001C01D92AE32B207CA
:100E3000E1F70E94BE100C94222F0C9400000FB614
:100E400080959AE0F8947BE27A95F1F708F0589A49
:100E500008F4589886959A95B1F70FBE08950FB685
:100E600080E8F894499BFECF4999FECF96E19A9588
:100E7000F1F79CE29A95F1F7869549998068C8F751
:100E80000FBE08950FB680E8F89496E19A95F1F7B1
:100E90009CE29A95F1F7869549998068C8F796E1A2
:100EA0009A95F1F7499BFECF0FBE0895FF93EF93FC
:100EB000E091A001F091A101309709F00995EF911F
:100EC000FF910895FC018591803011F0EFDFFBCF99
:100ED0000895FF27E0E230E247FF0CC0419597FFFD
:100EE00009C0EDE26095709580959095611D711D2A
:100EF000811D911D27FF02C0219530E350E2AA27F2
:100F0000660F771F881F991FAA1FA41710F0A41B34
:100F100063955A95A9F7AA3008F0A95FA05DAF9331
:100F2000F395611571058105910541F7ED3211F4D5
:100F3000EF93F395F21718F43F93F395FBCF8F914E
:100F4000B5DFFA95E1F70895E991F991859180303F
:100F500021F0853219F0AADFF9CF089520E0E89456
:100F600055915532C1F3503311F4689455915A3369
:100F700048F4505390F3220F022E220F220F200D1F
:100F8000250FF4CF0EF4219589919991533619F3D9
:100F9000533729F1533559F1BC0188279927E89433
:100FA0005C3621F48991999168945591543639F4BD
:100FB00046EF7EF077FF0DC08FEF9FEF0AC05537E9
:100FC0004AE039F0583540E121F0523642E009F06C
:100FD0000895FF93EF937DDFEF91FF91B7CFFF93DC
:100FE000EF93FC0181918030B9F360DFFBCFFF9379
:100FF000EF9368DFF1CFDF93CF93CDB7DEB72596C0
:10100000A3DFCF91DF91089514B88FEF85B9549A7B
:101010005C9808958FEF84B980E485B9549A5C9AFE
:101020008FE19EE40197F1F700C0000008958FEF73
:1010300084B980E485B957985F9A87B1806C87B985
:1010400088B1806C88B92E9A2F980E940408E2EB30
:10105000F1E080E18E0F11928E13FDCFE2EAF1E014
:1010600080E18E0F11928E13FDCF82EB91E0909371
:10107000C5018093C40182EA91E09093C3018093FB
:10108000C2010895EF92FF920F931F93CF93DF93C6
:101090008091C2019091C3012091C4013091C5019A
:1010A0003093C3012093C2019093C5018093C40182
:1010B0005C9B0E940A08C0E0D0E001E010E080E004
:1010C00090E0FC2FF770EC2FE87025B1207C2F2BDF
:1010D000AC0133E0440F551F3A95E1F7242B25B9B5
:1010E00028B12F73EE2311F0206401C0206828B9C5
:1010F0002AE12A95F1F700C0A091C201B091C30185
:10110000AC0FBD1F2C9130E0082E02C035952795FD
:101110000A94E2F720FD2F9AA5E3AA95F1F70000C3
:10112000F6B42E98BAE1BA95F1F700C04091C40127
:101130005091C501BA016C0F7D1F4F9B0BC09801E8
:10114000082E01C0220F0A94EAF72095DB013C919A
:10115000232309C0DB01EC909801082E01C0220F67
:101160000A94EAF72E292C9326B56F2D70E02F15DF
:1011700018F026B530E004C026B530E021503F4FCE
:10118000261B370B2630310558F0A091C201B091D3
:10119000C301AC0FBD1F2C91DA01AC0FBD1F2C9306
:1011A000BAE1BA95F1F700C02F982E9A20EA2A9555
:1011B000F1F701968830910509F087CFA091C4011D
:1011C000B091C501AC0FBD1FE091C201F091C30108
:1011D000EC0FFD1F9C918081981751F00E941926F9
:1011E0006093C6017093C7018093C8019093C901B1
:1011F0002196C031D10509F062CF5C9B1BC0809164
:101200002504853021F080912504811113C060915F
:10121000C6017091C7018091C8019091C9010E94D7
:101220004F26613177428105910520F00E94040824
:101230000E949A2581E0DF91CF911F910F91FF903D
:10124000EF9008952091C4013091C501F901E80F94
:10125000F11D808108950C940A080C940408569A94
:1012600081FF02C05E9A08955E98089588E0809399
:10127000CC001092CD00E9ECF0E0808180698083A1
:10128000808188608083EAECF0E080818083EBECF1
:10129000F0E080818083559A5D98789408959091CC
:1012A000CB012091CA019217D1F030E0F901E4534B
:1012B000FE4F80812F5F3F4F33272093CA01492F74
:1012C00050E0921718F4241B350B03C0241B350B78
:1012D0003395233031050CF05D9890E008958FEF41
:1012E0009FEF08959091C80095FFFCCF8093CE00AA
:1012F00008951F920F920FB60F9211242F933F93D0
:101300004F935F938F939F93EF93FF938091CB01C4
:1013100090E0AC014F5F5F4F2091CA01241741F06C
:101320003091CE00FC01E453FE4F30834093CB015B
:101330003091CB01822F90E0432F50E0841B950B1E
:10134000321708F0939503970CF45D9AFF91EF9193
:101350009F918F915F914F913F912F910F900FBE71
:101360000F901F9018958091E6020895089580913E
:10137000E60208950895089508950895CF93DF93A0
:101380008D3C9105B9F1B8F4853B9105A9F148F47C
:10139000833B9105D1F1843B9105D1F5D0E0C0E2CA
:1013A0003BC0873B910571F150F18C3C910581F573
:1013B000D0E0C8E031C08A3E9105C1F040F4823EE1
:1013C0009105B1F0893E910519F5D0E124C0813233
:1013D00022E0920749F0833222E09207D9F08A385E
:1013E0009140B1F4D2E017C0D4E015C0D0E213C0F0
:1013F000D0E411C0D0E80FC0D0E0C1E00DC0D0E013
:10140000C2E00AC0D0E0C4E007C0D0E0C0E104C040
:10141000D0E001C0D1E0C0E08DEF0E94720983E00E
:101420000E94720983E00E9472098D2F0E94720946
:101430008C2FDF91CF910C947209CF93DF93EC0145
:101440008DEF0E94720985E00E94720982E00E947D
:10145000720988810E94720989810E9472098A81B9
:101460000E9472098B81DF91CF910C947209CF9306
:10147000DF93EC018DEF0E94720989E00E947209EE
:1014800081E00E94720988810E94720980E00E94B6
:1014900072098A810E9472098B810E9472098C8173
:1014A0000E9472098D810E9472098E810E947209C8
:1014B0008F81DF91CF910C9472090C944F09EF92B8
:1014C000FF920F931F93CF938C010E940D267C01F6
:1014D000C0E0C7010E9425268017910798F40E945A
:1014E0004F099C012F3F8FEF380751F02D3041F00D
:1014F0002A3041F0EC2FF0E0E253FD4F2083CF5F24
:10150000C73138F3EC2FF0E0E253FD4F10828EEC40
:1015100092E0CF911F910F91FF90EF9008950C945E
:10152000720981B3881F8827881F0895879A8F9A28
:10153000089585B7806885BF85B7806885BF0E949C
:10154000960A86988E9A81988998559A5D980C94F7
:101550003609879A8F9808958FB18695817008957E
:101560008FB186FB882780F908958093E60208955D
:10157000CF93DF93FC018491EF012196882321F022
:101580000E947209FE01F7CFDF91CF910895CF93AA
:10159000DF93C2EFD1E00E944F098F3F2FEF9207F8
:1015A00059F09F938F93DF93CF930E94FB070F9087
:1015B0000F900F900F90EFCFDF91CF9108950E9481
:1015C000B80A2FEF89E698E1215080409040E1F77A
:1015D00000C0000084E690E00E945F0A8093CC0285
:1015E0009093CD029F938F9385EF91E09F938F937C
:1015F0000E94FB070E94C70A0F900F900F900F9058
:101600008091CC029091CD0208950E949E189093F3
:101610001501809314010E946A1E80E091E00E94EF
:1016200099180E94A90A0E94B00A8111FCCF8DE787
:1016300092E00E9462072FEF85EB95E321508040F6
:101640009040E1F700C0000089E792E00E94DF0AC5
:10165000EFEFFBE42DE1E150F0402040E1F700C066
:1016600000000E94C70A85E792E00E94DF0AFC01A1
:101670008081863721F081E792E00C94DF0A08959B
:1016800088E592E00E94620782E592E00E94DF0A0C
:101690000E94960A0E946A1E809114019091150181
:1016A0000C9499180E94FA0F8091210180932004D4
:1016B00008958F929F92AF92BF92CF92DF92EF9256
:1016C000FF920F931F93CF93DF9392E0B92E03EA1B
:1016D00014E029EAE22E24E0F22EAA24A39433E0B7
:1016E000932E41E9C42E44E0D42E0E945D0AEC0101
:1016F000019609F441C08091E9028130F9F028F0A7
:10170000823009F1833021F134C0CE3FD10519F484
:10171000A092E902EACFC038D10528F4DF93CF9335
:10172000FF92EF9204C0DF93CF931F930F930E9419
:10173000FB070F900F900F900F90D7CF2297C9F40F
:10174000B092E902D2CF2197A1F49092E902CDCFD5
:1017500080910F0480FF0AC0DF93CF93DF92CF9276
:101760000E94FB070F900F900F900F908C2F0E94FC
:10177000B50A1092E902B9CF8091EB02811127C01E
:101780008091EA02811114C00E94AC0A811110C03C
:101790000E949E188A509140D1F00E946A1E80914A
:1017A000210180932004109221018AE091E00DC074
:1017B0000E949E188651914051F00E946A1E8091AD
:1017C00020048093210186E191E00E949918809184
:1017D000E7029091E8020E942526893E23E09207C5
:1017E00008F461C028EE33E0B9010E94D22E629F56
:1017F000C001639F900D729F900D11242091E7020C
:101800003091E802820F931F9093E8028093E702E1
:101810000E949810833011F481E001C080E00E94A2
:10182000E90F0E94192628EE33E040E050E00E94C4
:10183000FA2E49015A018CE3C82ED12CE12CF12C4F
:10184000CA01B901A70196010E94FA2E672B682BE5
:10185000692B49F50E94611020910F0420FF23C0DD
:101860009F938F931F921F92C501B40120E13EE028
:1018700040E050E00E94FA2EC22FA70196010E947C
:10188000FA2E3F932F931F92CF938CE794E09F9370
:101890008F930E94FB078DB79EB70A960FB6F894F8
:1018A0009EBF0FBE8DBF0E94AC0A811107C00E946F
:1018B000B00A882319F06E9A769802C06E9A769ACA
:1018C000DF91CF911F910F91FF90EF90DF90CF901C
:1018D000BF90AF909F908F9008958F929F92AF92FC
:1018E000BF92CF92DF92EF92FF921F93CF93DF933D
:1018F00000D000D0CDB7DEB7833109F492C008F034
:1019000061C08B3009F46CC008F055C0853009F017
:1019100003C20E94192628EE33E040E050E00E9406
:10192000FA2E49015A010E9461109F938F938BEC0C
:1019300092E09F938F930E94FB07C501B40120E1C1
:101940003EE040E050E00E94FA2E5F934F933F93B9
:101950002F9325EC32E03F932F9369837A838B8317
:101960009C830E94FB078CE3C82ED12CE12CF12C28
:1019700069817A818B819C81A70196010E94FA2E50
:101980005F934F933F932F938FEB92E09F938F93AF
:101990000E94FB07C501B401A70196010E94FA2E1F
:1019A0009F938F937F936F9389EB92E09F938F9395
:1019B0000E94FB074AC18C3009F441C0813109F40F
:1019C000A4C1AAC1883361F020F4883109F443C16D
:1019D000A3C1873409F46AC18C3409F453C19CC192
:1019E00088E594E00E94620783E494E00E94620725
:1019F00089E294E00E94620782E094E00E9462071C
:101A000087EE93E00E94620785ED93E00E946207F3
:101A10001091EB02111111C085EB93E00E94620757
:101A20007FC10E94050B8DE992E00E94DF0A87E9E1
:101A300092E00E94DF0A0E94400B11E071C18CE924
:101A400093E00E9462070E949E188A50914019F00C
:101A500080E391E002C08AE291E09F938F938EE849
:101A600093E09F938F930E94FB078091EA021F925D
:101A70008F938FE793E09F938F930E94FB070E94C1
:101A8000AC0A0FB6F894DEBF0FBECDBF811107C000
:101A90000E94B00A811106C089E391E005C085E388
:101AA00091E002C08CE391E09F938F9385E793E0F0
:101AB0009F938F930E94FB070E94910A1F928F931E
:101AC0008AE593E09F938F930E94FB078091EB023E
:101AD0001F928F9389E493E09F938F930E94FB075B
:101AE000809125040FB6F894DEBF0FBECDBF8823CA
:101AF000B9F0809125048130B1F0809125048230C5
:101B0000A9F0809125048330A1F0809125048430D0
:101B100099F080912504853091F081E791E011C022
:101B200089E491E00EC081E491E00BC084E591E08E
:101B300008C08CE591E005C086E691E002C083E72D
:101B400091E09F938F938AE393E09F938F930E94FA
:101B5000FB0780E393E09F938F930E94FB070E9413
:101B600098100F900F900F900F900F900F90813062
:101B700059F038F0823059F0833061F48AE193E013
:101B80000BC08BE293E008C085E293E005C08EE1D4
:101B900093E002C088E193E09F938F930E94FB073C
:101BA0000F900F9086E193E09F938F930E94FB0725
:101BB000809123041F928F938DEF92E09F938F93D8
:101BC0000E94FB078091D90081701F928F9383EF51
:101BD00092E09F938F930E94FB070E94192628EEA4
:101BE00033E040E050E00E94FA2E69017A019CE364
:101BF000892E912CA12CB12CCA01B901A501940107
:101C00000E94FA2E7F936F93C701B60120E13EE058
:101C100040E050E00E94FA2E122FA50194010E948C
:101C2000FA2E3F932F931F921F93C701B60120E80E
:101C300031E541E050E00E94FA2E3F932F9386ED6C
:101C400092E09F938F930E94FB070FB6F894DEBF3C
:101C50000FBECDBFF2CE8091EB02811160C010911A
:101C6000EA02112339F08EEA92E00E946207109294
:101C7000EA0256C084EA92E00E94620781E0809303
:101C8000EA02DBCE0E94910A182F882341F00E94BD
:101C9000050B81E080931F048093EB0241C00E94FA
:101CA000400B10921F041092EB02C7CE8091EB0202
:101CB000811102C00E94050B8BE492E00E94DF0AB2
:101CC00080E492E00E94DF0A8CE292E00E94DF0A48
:101CD00085E292E00E94DF0A8BE192E00E94DF0A37
:101CE00084E192E00E94DF0A8AE092E00E94DF0A2B
:101CF00080E092E00E94DF0A8AEF91E00E94DF0A12
:101D00008091EB02811199CE96CE0E949E1811E02F
:101D10008651914029F403C01091EB0201C010E0FC
:101D2000812F0F900F900F900F90DF91CF911F9107
:101D3000FF90EF90DF90CF90BF90AF909F908F90EB
:101D40000895CF93C82F0E94CF24827291E009F4A6
:101D500090E04C2F50E0FA013497E934F10508F097
:101D6000D0C0EA5AFF4F0C941C2F8BE12DC191116A
:101D7000CCC081E629C19111CAC082E625C191116A
:101D8000C8C083E621C19111C6C084E61DC191116E
:101D9000C4C085E619C19111C2C086E615C1911172
:101DA000C0C087E611C19111BEC088E60DC1911176
:101DB000BCC089E609C19111BAC08AE605C191117A
:101DC000B8C08BE601C19111B6C08CE6FDC091117F
:101DD000B4C08DE6F9C09111B2C08EE6F5C0911184
:101DE000B0C08FE6F1C09111AEC080E7EDC0911197
:101DF000ACC081E7E9C09111AAC082E7E5C09111AA
:101E0000A8C083E7E1C09111A6C084E7DDC09111AD
:101E1000A4C085E7D9C09111A2C086E7D5C09111B1
:101E2000A0C087E7D1C091119EC088E7CDC09111B5
:101E30009CC089E7C9C091119AC08AE7C5C09111B9
:101E400098C081E3C1C0911196C082E3BDC09111D9
:101E500094C083E3B9C0911192C084E3B5C09111DD
:101E600090C085E3B1C091118EC086E3ADC09111E1
:101E70008CC087E3A9C091118AC088E3A5C09111E5
:101E800088C089E3A1C0911186C080E39DC088E02D
:101E90009BC089E099C080E297C091117EC08DE21D
:101EA00093C091117CC08DE38FC091117AC08BE5F6
:101EB0008BC0911178C08DE587C0992309F475C056
:101EC0008CE782C0992309F472C08CE77DC0911120
:101ED00070C08BE379C091116EC087E275C091111B
:101EE0006CC080E671C091116AC08CE26DC0911126
:101EF00068C08EE269C0911166C08FE265C080E063
:101F000063C080E261C08AE05FC081E45DC082E4BA
:101F10005BC083E459C084E457C085E455C086E4BF
:101F200053C087E451C088E44FC089E44DC08AE4BF
:101F30004BC08BE449C08CE447C08DE445C08EE4BF
:101F400043C08FE441C080E53FC081E53DC082E5EC
:101F50003BC083E539C084E537C085E535C086E5FB
:101F600033C087E531C088E52FC089E52DC08AE5FB
:101F70002BC081E229C080E427C083E225C084E22F
:101F800023C085E221C08EE51FC086E21DC08AE223
:101F90001BC088E219C089E217C08FE515C08BE22B
:101FA00013C08BE711C08DE70FC08CE50DC08CE529
:101FB0000BC08AE309C082E207C08EE705C08CE34C
:101FC00003C08EE301C08FE30E948F0A81E0CF91AE
:101FD0000895833019F4859A7D9A0895813011F41B
:101FE000859A06C0823019F4859A8D9A089585984D
:101FF0008D98089581E00E94E90F2FEF81EE94E023
:10200000215080409040E1F700C0000082E00E9433
:10201000E90F2FEF81EE94E0215080409040E1F7EE
:1020200000C0000081E00E94E90F2FEF81EE94E0F4
:10203000215080409040E1F700C0000082E00E9403
:10204000E90F2FEF81EE94E0215080409040E1F7BE
:1020500000C0000080E00E94E90F80EC80937C00CB
:1020600087E080937A0081E980937E0081E080930D
:102070007F008BE380937D00849A8C9808958091F3
:10208000D90080FF1CC090B331B385988D9AEFE9D9
:10209000FFE03197F1F700C000008FB185FB882782
:1020A00080F920B390722F7D292B20BB91B3232F71
:1020B00020729F7D922B91BB91E08927089580E04B
:1020C0000895CF93DF9300D0CDB7DEB7849A8C9A72
:1020D00080917A00806880937A008FE99FE0019771
:1020E000F1F700C0000080917A00806480937A004C
:1020F00080917A0086FDFCCF8091780090917900E4
:102100009A83898380917A008F7780937A00849A6A
:102110008C9829813A8145E0429FC001439F900DF0
:102120001124805591090F900F90DF91CF91089560
:102130008091D90080FD0C943F100E9461108C3A70
:102140002DE0920720F481E08093EC0205C08537F2
:102150009E4010F01092EC028091EC02811102C0BE
:1021600082E0089583E00895CF93C82F0E941F074F
:102170008C2F0E94361180E0CF91089584B7877F1D
:1021800084BF0FB6F894A895809160008861809311
:102190006000109260000FBE90E080E80FB6F894E7
:1021A00080936100909361000FBE0E94B7150E945A
:1021B00014168091E20084608093E20084EB90E149
:1021C0000E946B25509A589A5198599A78948FEF9B
:1021D000909125048150943041F0EFE7FEE3319770
:1021E000F1F700C000008111F3CF8CEC94E00E9465
:1021F00062070E94990A0E94520B80EC94E00E94B0
:1022000062070E945F1980EB94E00E9462070E94BF
:10221000AC0A882319F1809125048530F9F48CEA01
:1022200094E00E9462070E942D090E949A250E9454
:102230009A250E949A250E949A250E949A250E941A
:102240009A250E949A2580912304882301F30E94F5
:10225000C3258823E1F20E940C14D9CF0E94631990
:102260000E94590BD4CF8091110308959FB7F89421
:102270001092F0029FBF90912504943009F057C04E
:102280009091E9009F703091EC00232F217030FD78
:1022900020E8922B24E02093E9002091EB0020FF1E
:1022A00043C02091EE0027FF3FC02091ED02222382
:1022B00021F02091E80025FF37C01092ED0226E0C2
:1022C0003091E80035FD15C030912504343061F5BA
:1022D0003091EB0035FD28C0215021F481E080933E
:1022E000ED0222C0EFE9FFE03197F1F700C00000F6
:1022F000E7CF8093F1008091E80085FD0AC08091CE
:10230000E80080FFFCCF8091E8008E778093E800A2
:1023100006C08FB7F89421E02093F0028FBF9F7022
:102320009093E90080E008959F709093E9008FEF0B
:102330000895CF93DF9300D01F92CDB7DEB79C01F5
:1023400080912504843019F593E099833B832A8397
:102350009093E9008FEF9091E800815095FD06C0C1
:1023600095ED9A95F1F700008111F5CF8091E80085
:1023700085FF0DC040E050E063E070E0CE010196C3
:102380000E9422148091E8008E778093E8000F90DD
:102390000F900F90DF91CF910895CF93DF9300D0EE
:1023A0001F92CDB7DEB720912504243021F522E01D
:1023B00029839B838A8383E08093E9008FEF909148
:1023C000E800815095FD06C095ED9A95F1F7000063
:1023D0008111F5CF8091E80085FF0DC040E050E00D
:1023E00063E070E0CE0101960E9422148091E80023
:1023F0008E778093E8000F900F900F90DF91CF9130
:102400000895209125042430F1F422E02093E9007E
:102410002FEF3091E800215035FD06C035ED3A959B
:10242000F1F700002111F5CF2091E80025FF0BC046
:1024300040E050E065E070E00E9422148091E800E6
:102440008E778093E8000895CF93DF932091250441
:10245000243009F048C0EC01809120018823E1F08C
:10246000809121018823C1F085E08093E9008FEFFE
:102470009091E800815095FD06C09AE29A95F1F797
:1024800000C08111F5CF8091E80085FF2CC040E0AD
:1024900050E060E270E017C081E08093E9008FEFC8
:1024A0009091E800815095FD06C095ED9A95F1F761
:1024B00000008111F5CF8091E80085FF14C040E055
:1024C00050E068E070E0CE010E9422148091E800A4
:1024D0008E778093E80080E2FE01A1EFB2E00190E8
:1024E0000D928A95E1F7DF91CF9108958BED94E0FD
:1024F0000E94620780912404811109C00E94B715CF
:102500000E9414168091E20084608093E200089596
:1025100087ED94E00E9462071092240408950895C4
:102520002091EE022F5F822F62E30E94C62E992334
:1025300019F02093EE0208951092EE028091F002BD
:10254000882371F180912504843041F58091E90060
:102550008F702091EC00922F917020FD90E8892BD4
:1025600094E09093E9009091EB0090FF14C090915B
:10257000EE0097FF10C09091E80095FF03C0109205
:10258000F100F9CF9091E80090FF05C09091E8002C
:102590009E779093E8008F708093E9001092F0028C
:1025A000089542E061EC81E00E94311542E061EC67
:1025B00082E00E94311542E061EC83E00E94311517
:1025C00042E261EC84E00E94311542E261EC85E078
:1025D0000C94311580912704833009F455C030F4F0
:1025E000813071F0823009F48EC008958A3009F488
:1025F0007AC08B3009F460C0893009F09CC020C0DB
:1026000080912604813A09F096C08091E800877F86
:102610008093E80080912A0490912B04892B21F467
:1026200060E281EF92E003C060E080E090E070E063
:102630000E946D148091E8008B778093E8000895E4
:1026400080912604813209F076C080912A0490910D
:102650002B04009719F0049709F06DC08091E800F1
:10266000877F8093E8008091E80082FD05C080911B
:1026700025048111F8CF5FC08091F1008093110390
:102680008091E8008B7753C080912604813A09F04D
:1026900052C080912A0490912B04892B09F04BC0E1
:1026A0008091E800877F8093E8008091E80080FFB8
:1026B000FCCF8091200136C0809126048132D9F56B
:1026C00080912A0490912B04892BA9F58091E80030
:1026D000877F8093E8000E9466158091280480938C
:1026E00020010C946A1E80912604813221F580918C
:1026F000E800877F8093E8000E9466158091290496
:1027000080931203089580912604813AA1F4809168
:10271000E800877F8093E8008091E80080FFFCCF8D
:10272000809112038093F1008091E8008E7780936E
:10273000E8000C9466150895809111038093EF02D0
:102740001092110380E00E942F090E94081A0C9435
:102750006A1E0C949C130E94D7258091EF028093EF
:10276000110308950C94AB13292F3327233031051F
:10277000C9F064F42130310581F02230310509F0CF
:1027800043C08DE890E027E035E042C021323105BA
:10279000F1F02232310541F137C082E190E024E9C5
:1027A00035E036C099278130910541F0823091059E
:1027B00041F0892B49F5E3E0F5E005C0E3EFF4E0F3
:1027C00002C0EFEDF4E0849190E09F0121C06530FC
:1027D000D8F4E62FF0E0EE0FFF1FE457FE4F208104
:1027E000318189E090E014C0653070F470E0FB0145
:1027F000EE0FFF1FEE57FE4F20813181FB01E358A2
:10280000FE4F808190E004C080E090E020E030E066
:10281000FA0131832083089580E189BD82E189BD79
:1028200009B400FEFDCF8091D8008F7D8093D80041
:102830008091E00082608093E0008091E00081FD63
:10284000FCCF0895CF92DF92EF92FF920F931F93E8
:10285000CF93DF93EC018B016A010E9485158111F2
:1028600033C0C114D10439F0F60180819181081B75
:10287000190BC80FD91FE12CF12C0115110519F105
:102880008091E80085FD16C08091E8008E778093E6
:10289000E800C114D10449F0F60180819181E80E6D
:1028A000F91EF182E08285E00FC00E948515882321
:1028B00021F30AC089918093F10001501109FFEFC3
:1028C000EF1AFF0ADACF80E0DF91CF911F910F91CD
:1028D000FF90EF90DF90CF90089520912C043091DD
:1028E0002D042617370748F06115710539F420913A
:1028F000E8002E772093E80001C0B90140E061159F
:102900007105A9F120912504222309F443C0253043
:1029100009F442C02091E80023FD40C02091E80066
:1029200022FD32C02091E80020FFE9CF4091F30062
:102930002091F20030E0342BFC01CF0161157105CC
:1029400059F02830310540F481918093F1006150B5
:1029500071092F5F3F4FF1CF41E02830310509F079
:1029600040E02091E8002E772093E800C8CF411185
:10297000C9CF0AC080912504882361F0853061F0B9
:102980008091E80083FD0AC08091E80082FFF2CFC9
:1029900080E0089582E0089583E0089581E008953D
:1029A00020912C0430912D042617370748F061152B
:1029B000710539F42091E8002E772093E80001C0DA
:1029C000B901FC0120E06115710591F180912504A8
:1029D000882309F440C0853009F43FC08091E800A5
:1029E00083FD3DC08091E80082FD2FC08091E8000A
:1029F00080FFE9CF2091F3008091F20090E0922BCC
:102A00006115710559F08830910540F424912093A7
:102A1000F1003196615071090196F2CF21E00897DB
:102A200009F020E08091E8008E778093E800CBCF1A
:102A30002111CCCF0AC080912504882361F0853014
:102A400061F08091E80083FD0AC08091E80082FF78
:102A5000F2CF80E0089582E0089583E0089581E058
:102A60000895982F973058F59093E900981739F00A
:102A70007091EC002091ED005091F00003C0242FE4
:102A8000762F50E021FF19C03091EB003E7F30934C
:102A9000EB003091ED003D7F3093ED003091EB0085
:102AA00031603093EB007093EC002093ED00509375
:102AB000F0002091EE0027FF07C09F5FD3CF8F70FB
:102AC0008093E90081E0089580E0089580912604D4
:102AD00087FF11C08091E80082FD05C08091250428
:102AE0008111F8CF11C08091E8008B770BC08091E5
:102AF0002504882349F08091E80080FFF8CF809179
:102B0000E8008E778093E80008952091E4003091EA
:102B1000E50095E64091EC00842F817040FF22C0D3
:102B20008091E80080FD1CC080912504882391F0ED
:102B3000853091F08091EB0085FD10C04091E4005C
:102B40005091E5004217530729F39A01915011F76C
:102B500084E0089582E0089583E0089581E0089577
:102B600080E008954091E80042FFDECF08950E9482
:102B700025160E942D16E0EEF0E0808181608083B2
:102B8000E8EDF0E080818F77808319BCA7EDB0E09D
:102B90008C918E7F8C9380818F7E80831092240411
:102BA00008950F931F93CF93DF930E9425160E94E1
:102BB0002D16C8EDD0E088818F7788838881806862
:102BC000888388818F7D888319BC10922504109298
:102BD0002104109223041092220400EE10E0F80168
:102BE00080818B7F808388818160888342E060E080
:102BF00080E00E943115E1EEF0E080818E7F8083DD
:102C0000E2EEF0E080818160808380818860808353
:102C1000F80180818E7F8083888180618883DF9145
:102C2000CF911F910F910895E8EDF0E080818F7EA4
:102C30008083E7EDF0E080818160808384E082BF63
:102C400081E0809324040C94D115E8EDF0E08081BC
:102C50008E7F80831092E20008951092DA00109225
:102C6000E10008951F920F920FB60F9211242F9337
:102C70003F934F935F936F937F938F939F93AF9304
:102C8000BF93EF93FF938091E10082FF0BC080918F
:102C9000E20082FF07C08091E1008B7F8093E1001A
:102CA0000E9490128091DA0080FF1FC08091D800AE
:102CB00080FF1BC08091DA008E7F8093DA008091C4
:102CC000D90080FF0DC080E189BD82E189BD09B4D2
:102CD00000FEFDCF81E0809325040E94761205C09E
:102CE00019BC109225040E9488128091E10080FF97
:102CF00019C08091E20080FF15C08091E2008E7FB4
:102D00008093E2008091E20080618093E2008091F4
:102D1000D80080628093D80019BC85E08093250498
:102D20000E94A9138091E10084FF30C08091E200ED
:102D300084FF2CC080E189BD82E189BD09B400FE19
:102D4000FDCF8091D8008F7D8093D8008091E100E5
:102D50008F7E8093E1008091E2008F7E8093E2007D
:102D60008091E20081608093E200809121048823B9
:102D700011F084E007C08091E30087FD02C081E08C
:102D800001C083E0809325040E94B2138091E1008A
:102D900083FF29C08091E20083FF25C08091E1007C
:102DA000877F8093E10082E08093250410922104C4
:102DB0008091E1008E7F8093E1008091E2008E7F20
:102DC0008093E2008091E20080618093E20042E023
:102DD00060E080E00E9431158091F000886080936F
:102DE000F0000E948F12FF91EF91BF91AF919F91E0
:102DF0008F917F916F915F914F913F912F910F90A4
:102E00000FBE0F901F9018951F920F920FB60F9242
:102E100011242F933F934F935F936F937F938F93DF
:102E20009F93AF93BF93CF93DF93EF93FF93C091A3
:102E3000E900CF708091EC00D82FD17080FDD0E8F0
:102E40001092E9008091F000877F8093F0007894E1
:102E50000E9448171092E9008091F00088608093EA
:102E6000F000CD2BCF70C093E900FF91EF91DF917F
:102E7000CF91BF91AF919F918F917F916F915F9112
:102E80004F913F912F910F900FBE0F901F9018956B
:102E90001F93CF93DF93CDB7DEB7AA970FB6F89401
:102EA000DEBF0FBECDBFE6E2F4E088E08E0F90916A
:102EB000F10091938E13FBCF0E94EA128091E800FB
:102EC00083FF1FC18091260490912704492F50E071
:102ED0004A30510508F015C1FA01E156FF4F0C9434
:102EE0001C2F803881F0823809F00BC180912A04B0
:102EF0008F708093E9008091EB0085FB882780F933
:102F00001092E90006C0809122049091230491114F
:102F100082609091E800977F9093E8008093F100A1
:102F20001092F100C8C0282F2D7F09F0EAC0882335
:102F300019F0823061F0E5C080912804813009F0F9
:102F4000E0C0933009F080E0809323042BC080918F
:102F50002804811127C080912A048F7009F4D1C000
:102F60008093E9002091EB0020FF1CC0933021F4F6
:102F70008091EB00806214C09091EB00906190937F
:102F8000EB0021E030E0A90102C0440F551F8A95F3
:102F9000E2F74093EA001092EA008091EB0088602B
:102FA0008093EB001092E9008091E800877F86C053
:102FB0008111A7C0109128041F778091E3008078C9
:102FC000812B8093E3008091E800877F8093E80065
:102FD0000E9466158091E80080FFFCCF8091E3009D
:102FE00080688093E300111102C082E001C083E099
:102FF0008093250486C08058823008F082C080917A
:103000002804909129048C3D53E0950779F583E0DD
:103010008A838AE289834FB7F894DE01139620E011
:103020003EE051E2E32FF0E050935700E49120FF9F
:1030300003C0E295EF703F5FEF708E2F90E0EA30B3
:1030400010F0C79601C0C0968D939D932F5F2431D9
:1030500049F74FBF8091E800877F8093E8006AE2DC
:1030600070E0CE0101960E946D1414C0AE014F5F56
:103070005F4F60912A040E94B413BC01892B09F4AC
:1030800040C09091E800977F9093E80089819A81F1
:103090000E94D0148091E8008B778093E80031C0C3
:1030A000803879F58091E800877F8093E8008091EF
:1030B00021048093F1008091E8008E778093E800EE
:1030C0000E9466151EC081111CC090912804923088
:1030D000C0F48091E800877F8093E80090932104FA
:1030E0000E94661580912104811106C08091E30041
:1030F00087FD02C081E001C084E0809325040E9426
:10310000D1128091E80083FF0AC08091E800877F98
:103110008093E8008091EB0080628093EB00AA9698
:103120000FB6F894DEBF0FBECDBFDF91CF911F91D8
:1031300008959093180380931703089580911703BF
:10314000909118030895E0911703F09118033097B8
:1031500021F00190F081E02D099480E00895EF9234
:10316000FF920F931F93CF93DF93E0911703F0919A
:1031700018033097B1F18C010280F381E02D09959D
:1031800080910F0482FF2DC080FF04C08AEE96E07C
:103190000E946207E80110E284EEE82E86E0F82E35
:1031A00080910F0480FF0BC088811F928F93FF9244
:1031B000EF920E94FB070F900F900F900F9011500D
:1031C00021961111EDCF80910F0480FF0AC082EE8D
:1031D00096E0DF91CF911F910F91FF90EF900C94AB
:1031E0006207DF91CF911F910F91FF90EF900895AB
:1031F000E0911703F0911803309721F00480F581D6
:10320000E02D09940895CF93DF93EC01809115038D
:1032100090911603C817D90709F1D0931603C093EC
:103220001503E0911703F09118033097B9F0068069
:10323000F781E02DCE01099580910F0482FF0EC029
:1032400080FF0CC0DF93CF9384ED96E09F938F9324
:103250000E94FB070F900F900F900F90DF91CF917E
:103260000895CF93DF93EC018091130390911403A1
:10327000C817D90709F1D0931403C0931303E09141
:103280001703F09118033097B9F00084F185E02D11
:10329000CE01099580910F0482FF0EC080FF0CC003
:1032A000DF93CF9384EC96E09F938F930E94FB076C
:1032B0000F900F900F900F90DF91CF9108950E9483
:1032C00004260C941708BF92CF92DF92EF92FF92E0
:1032D0000F931F93CF93DF9300D000D01F92CDB7F1
:1032E000DEB70E9442080AE113E0F12C8F2D0E9404
:1032F0002209B82EF801C080C82639F4F3940F5F74
:103300001F4FF0E1FF12F2CF30C080910F0481FD1A
:103310000E94091AD12CEE24E3948E2D8C21F9F011
:10332000D982FA8281E09E2D9B2109F480E08B8373
:103330000E940D268160782F9D838C8349815A815C
:103340006B818D810E943D1A49815A816B817C81FC
:103350008D810E948725F80190819E259083D394CA
:10336000EE0CF8E0DF12D9CFC9CF8FEF89838A83C3
:103370001B820E940D268160782F9D838C8349815A
:103380005A816B818D810E943D1A0E9486250E9480
:10339000FA28109119030E94A318181741F10E94EE
:1033A000A3188093190390910F0492FF0EC090FF11
:1033B0000CC01F928F9385EF96E09F938F930E948E
:1033C000FB070F900F900F900F90809119030F90B3
:1033D0000F900F900F900F90DF91CF911F910F9151
:1033E000FF90EF90DF90CF90BF900C9498250F90B6
:1033F0000F900F900F900F90DF91CF911F910F9131
:10340000FF90EF90DF90CF90BF9008950C942F091C
:103410000895EF92FF920F931F93CF93DF938EE067
:1034200097E00E946207C0E0D0E08FE2E82E81E0E2
:10343000F82E00E017E08C2F0E9422090E947025D0
:10344000FF92EF921F928F93DF93CF931F930F936F
:103450000E94FB0721968DB79EB708960FB6F89489
:103460009EBF0FBE8DBFC031D10529F7DF91CF912F
:103470001F910F91FF90EF900895CF93DF93CDB7F9
:10348000DEB72B970FB6F894DEBF0FBECDBF942FDB
:103490004F83252F588769877A878B874A855B8575
:1034A000452B21F02F3F09F59F3FF9F4DE011196DE
:1034B00086E0FD0111928A95E9F785E0FE013796D5
:1034C00001900D928A95E1F749815A816B817C8147
:1034D0008D819E810E944F212B960FB6F894DEBFFE
:1034E0000FBECDBFDF91CF9108954F81588569857B
:1034F0007A858B850E948725D9CFCF93882309F4BD
:1035000065C0C82F8CEF8C0F813A20F080E58C0FBE
:103510008E3248F48C2F0E94402C811157C08C2F82
:103520000E9427240CC080E28C0F883058F4C770AA
:1035300081E001C0880FCA95EAF70E94D224CF919A
:103540000C9416258BE58C0F833078F4C53A29F05E
:10355000C63A31F083E890E005C081E890E002C00F
:1035600082E890E0CF910C94031988E58C0F8531A7
:1035700068F5C83A89F0C93A91F0CA3A99F0CB3A5D
:10358000A1F0CC3AA9F0CD3AB1F0CE3AB9F0CF3AA9
:10359000C1F080E090E017C082EE90E014C089EEA8
:1035A00090E011C08AEE90E00EC085EB90E00BC079
:1035B00086EB90E008C083EB90E005C084EB90E0E0
:1035C00002C087EB90E0CF910C943119CF91089510
:1035D000882349F19CEF980F913A20F090E5980FDD
:1035E0009E3218F40E947A240DC090E2980F983011
:1035F00058F4877091E001C0990F8A95EAF7892FF6
:103600000E94D8240C9416259BE5980F933020F443
:1036100080E090E00C940319885A853120F480E012
:1036200090E00C9431190895882321F00E94D2244F
:103630000C9416250895882321F00E94D8240C9418
:1036400016250895BF92CF92DF92EF92FF920F93CB
:103650001F93CF93DF9300D000D000D0CDB7DEB75B
:1036600025E0FC01DE01119601900D922A95E1F70B
:10367000FC01408151810281638174812581229501
:103680002F706115710509F403C35F3F19F44F3FB3
:1036900009F4FEC26C01862F7D836C83602F782F26
:1036A0008D812E830E94AB23182FB92E0E94AA234E
:1036B0000E949A22EB2DE295EF70F0E0E755FF4F64
:1036C0002E810C941C2F8B2D807F9B2D9F70F92EAB
:1036D000882319F0F29490EFF922002349F0FF209B
:1036E00009F483C28F2D0E94E5240E9416257DC215
:1036F000812F0E94E81AFF2009F4CAC28F2D0E9470
:10370000EB2426960FB6F894DEBF0FBECDBFDF9137
:10371000CF911F910F91FF90EF90DF90CF90BF90CE
:103720000C9416258B2D807F9B2D9F70F92E803257
:1037300019F0F29480EFF822112319F0113009F1F9
:103740002AC00023B1F08F2D222351F1213041F501
:1037500026960FB6F894DEBF0FBECDBFDF91CF9196
:103760001F910F91FF90EF90DF90CF90BF900C943E
:10377000F524222319F0213009F48AC20E94FE2484
:103780002DC00023F1F0263008F082C20E94CF2421
:103790008F2129F023C00023F9F0211116C08F2DAD
:1037A00026960FB6F894DEBF0FBECDBFDF91CF9146
:1037B0001F910F91FF90EF90DF90CF90BF900C94EE
:1037C000141B253008F064C209C0F601858180FF12
:1037D0000CC28F708583E3CF21111CC28F2D83C152
:1037E0002B2D26952695237030E02115310521F0EB
:1037F00021303105D1F04CC2002321F0812F9B2DC7
:10380000937002C080E090E026960FB6F894DEBF79
:103810000FBECDBFDF91CF911F910F91FF90EF9021
:10382000DF90CF90BF900C940319002321F0812FDB
:103830009B2D937002C080E090E026960FB6F8941E
:10384000DEBF0FBECDBFDF91CF911F910F91FF90D3
:10385000EF90DF90CF90BF900C943119812F00230F
:1038600019F00E94802702C00E94E82726960FB612
:10387000F894DEBF0FBECDBFDF91CF911F910F91A6
:10388000FF90EF90DF90CF90BF900C946D288B2D20
:10389000837009F07BC00111FBC1812F8295869551
:1038A0008770880F880F912F9F70C92ED12CE12C23
:1038B000F12C082E04C0CC0CDD1CEE1CFF1C0A945D
:1038C000D2F714FF12C04FE050E060E070E004C097
:1038D000440F551F661F771F8A95D2F7CB01BA0197
:1038E000609570958095909503C060E070E0CB0185
:1038F0002B2D269526952370422F50E042305105FE
:10390000D9F04330510569F16C297D298E299F2911
:103910004130510551F126960FB6F894DEBF0FBE27
:10392000CDBFDF91CF911F910F91FF90EF90DF906E
:10393000CF90BF900C94BF226C297D298E299F299E
:1039400026960FB6F894DEBF0FBECDBFDF91CF91A4
:103950001F910F91FF90EF90DF90CF90BF900C944C
:10396000D9220E94BF22C701B60126960FB6F8944D
:10397000DEBF0FBECDBFDF91CF911F910F91FF90A2
:10398000EF90DF90CF90BF900C94A522002319F008
:103990008B2D817001C08695882309F479C1812F10
:1039A000829586958770880F880F912F9F70C92EFA
:1039B000D12CE12CF12C082E04C0CC0CDD1CEE1C0B
:1039C000FF1C0A94D2F714FF12C04FE050E060E0F1
:1039D00070E004C0440F551F661F771F8A95D2F709
:1039E000CB01BA01609570958095909503C060E019
:1039F00070E0CB012B2D269526952370422F50E0A9
:103A000042305105D9F04330510569F16C297D29C7
:103A10008E299F294130510551F126960FB6F89411
:103A2000DEBF0FBECDBFDF91CF911F910F91FF90F1
:103A3000EF90DF90CF90BF900C9486236C297D2966
:103A40008E299F2926960FB6F894DEBF0FBECDBFF4
:103A5000DF91CF911F910F91FF90EF90DF90CF906A
:103A6000BF900C9498230E948623C701B601269626
:103A70000FB6F894DEBF0FBECDBFDF91CF911F917F
:103A80000F91FF90EF90DF90CF90BF900C94742334
:103A9000103FD1F128F480E4810F803250F0A0C0B3
:103AA000123F09F462C008F44BC0133F09F472C01E
:103AB00097C0F12FF071FF2E8B2D8F71002351F0E5
:103AC0000E940D23812FFF2019F08295807F68CE00
:103AD0008F7066CE0E942E23812FFF2019F08295D1
:103AE000807F01C08F7026960FB6F894DEBF0FBEA0
:103AF000CDBFDF91CF911F910F91FF90EF90DF909D
:103B0000CF90BF900C941B1B0023B1F0253008F020
:103B1000BFC08B2D8F7126960FB6F894DEBF0FBEF7
:103B2000CDBFDF91CF911F910F91FF90EF90DF906C
:103B3000CF90BF900C945323263008F0A9C0E9CF52
:103B40000023A9F08B2D8F7126960FB6F894DEBF57
:103B50000FBECDBFDF91CF911F910F91FF90EF90DE
:103B6000DF90CF90BF900C940D23002359F38B2D41
:103B70008F7126960FB6F894DEBF0FBECDBFDF91D2
:103B8000CF911F910F91FF90EF90DF90CF90BF905A
:103B90000C942E23002399F08B2D8F7126960FB64F
:103BA000F894DEBF0FBECDBFDF91CF911F910F9173
:103BB000FF90EF90DF90CF90BF900C94F822269664
:103BC0000FB6F894DEBF0FBECDBFDF91CF911F912E
:103BD0000F91FF90EF90DF90CF90BF900C94F32265
:103BE0000023A9F0222309F4ADCF812F26960FB62A
:103BF000F894DEBF0FBECDBFDF91CF911F910F9123
:103C0000FF90EF90DF90CF90BF900C947D1A22230D
:103C100009F4ADCF812F26960FB6F894DEBF0FBE04
:103C2000CDBFDF91CF911F910F91FF90EF90DF906B
:103C3000CF90BF900C94E81A4B2D4F70612FC601A6
:103C40000E94FA2626960FB6F894DEBF0FBECDBFAF
:103C5000DF91CF911F910F91FF90EF90DF90CF9068
:103C6000BF900C94F3214B2D4F70612FC601269607
:103C70000FB6F894DEBF0FBECDBFDF91CF911F917D
:103C80000F91FF90EF90DF90CF90BF900C94FD26A6
:103C900026960FB6F894DEBF0FBECDBFDF91CF9151
:103CA0001F910F91FF90EF90DF90CF90BF900895FC
:103CB0000E94F2240E94C1240E9416250E949F297E
:103CC0000E946D2880E090E00E94031980E090E05F
:103CD0000C9431190E94E2240C94581ECF93DF9368
:103CE00000D000D01F92CDB7DEB7942F4983252F87
:103CF0005A836B837C838D834C815D81452B39F1A5
:103D00002F3F11F49F3F19F149815A816B817C81CA
:103D10008D810E94AB23292F22952F7030E02C300B
:103D2000310504F52A3031055CF422503109223086
:103D3000310568F4853A80F4843090F4823080F064
:103D4000883E38F4803E60F48450813A48F080E048
:103D500014C0803FE1F704C090E2980F983080F7DC
:103D600081E00BC02C30310521F493FB882780F9CA
:103D700004C02F303105C9F3EACF0F900F900F9098
:103D80000F900F90DF91CF910895CF93DF9300D0E4
:103D900000D01F92CDB7DEB70F900F900F900F900D
:103DA0000F90DF91CF910895CF93DF9300D000D093
:103DB00000D0CDB7DEB726960FB6F894DEBF0FBEA3
:103DC000CDBFDF91CF9108951F93CF93DF93C09123
:103DD0002A0316E080912B03C81799F0D0E01C9FAE
:103DE000F0011D9FF00D1124E45DFC4F40815181D5
:103DF00062817381848195810E94D41E2196C7704F
:103E0000E9CFDF91CF911F91089540915C035091CC
:103E10005D0360915E0370915F03809160039091F8
:103E200061030C94D41E8091610382958F7009F018
:103E300054C080915E03882309F44FC080912A0307
:103E4000A0912B0360915C0370915D0340915F032F
:103E500050916003B6E08A1709F43FC090E0411525
:103E60005105C1F17F3F11F46F3FA1F1B89FF001FF
:103E7000B99FF00D1124E45DFC4F218172132AC01B
:103E80002081621327C02281211124C02381348123
:103E90002417350710F421503109241B350B2C321F
:103EA0003140C0F4209161032F70206120936103A1
:103EB00026E0289FF001299FF00D1124EF5CFC4FB4
:103EC00080818F70806180838CE593E00E94221B4B
:103ED0000C94E41E01968770BECF0895BF92CF92D6
:103EE000DF92EF92FF920F931F93CF93DF93CDB7A3
:103EF000DEB761970FB6F894DEBF0FBECDBF7C0171
:103F000085E0F701DE011D9601900D928A95E1F79B
:103F1000D7014C9111965C9111971296DC901297F3
:103F200013960D911C91149730915C0360915D0381
:103F300080915F0390916003009709F47FC16F3F08
:103F400019F43F3F09F47AC1B0905E03BB2009F435
:103F5000CAC0209161030817190750F0F801E81B47
:103F6000F90BCF01CC24C3948C329140D0F009C01E
:103F700080959095800F911FCC24C3948C329140F2
:103F800080F0C12C207F09F0CCC0702F198B088BDA
:103F90006D2D89890E94C51E8CE593E00E94221B2D
:103FA000B6C0822F807F09F047C0651314C0341358
:103FB00012C0D11010C02F702061209361030E94A5
:103FC000051F8CE593E00E94221B80916103D701BD
:103FD00015968C932FC00115110519F15F3F11F44F
:103FE0004F3FF9F0CD2CD1101CC080912A032091B5
:103FF0002B0336E0821709F45CC090E0389FF00193
:10400000399FF00D1124E45DFC4F6181561306C009
:104010006081461303C06281611103C001968770FD
:10402000E9CFCD2CDD2009F429C1809161038160A5
:1040300080936103C12C22C1651308C0341306C0EC
:10404000D11004C080916103D701CCC04D875E8739
:10405000DF86702F198B088B6D2D89890E946E1E4B
:104060008823E9F1DD20D9F120916103822F829527
:104070008F7090E0029774F080915C0390915D03E3
:1040800098878F8319861B870A872C87CE0107960E
:104090000E94221B86E0F701ACE5B3E001900D928F
:1040A0008A95E1F70E94131F0E94051FCC24C39438
:1040B000E5C0702F198B088B60E089890E94AB23C3
:1040C000292F22952F7030E0223031050CF0CAC024
:1040D0009F7009F0C4C0805E883008F4CFC0C7016B
:1040E0000E94221BE3CF0817190708F456C0F801F5
:1040F000E81BF90BCF018C32914008F456C0C12C5B
:10410000702F198B088B6D2D89890E94C51EECE5D7
:10411000F3E086E0DF011D928A95E9F70E94051F12
:10412000ADC0651314C0341312C0D11010C08091FB
:104130006103F7018583C7010E94221B86E0ECE53D
:10414000F3E0DF011D928A95E9F7CB2C97C04D87EC
:104150005E87DF86702F198B088B6D2D89890E94F1
:104160006E1E882309F4BBCFDD2009F4B8CF20915F
:104170006103822F82958F7090E002970CF48ACFB2
:1041800080915C0390915D039A8389831B821D83D8
:104190000C832E83CE0101967BCF80959095800F66
:1041A000911F8C32914008F0AACFCD2CDD2009F46C
:1041B00096CF65132EC034132CC02091610320FDCF
:1041C0001FC0822F82958F70D9F0D70115962C933E
:1041D00015978F3049F08F5F982F9295907F822F9F
:1041E0008F70892B15968C93C7010E94221B86E045
:1041F000F701ACE5B3E001900D928A95E1F78ECF1F
:1042000086E0F701ACE5B3E001900D928A95E1F705
:1042100035C04D875E87DF86702F198B088B6D2D1B
:1042200089890E946E1E811135CF80916103816062
:1042300080936103C7010E94221B20C0DD2009F486
:104240004ECF4D875E87DF86702F198B088B6D2DC3
:1042500089890E946E1E882309F441CF1BCF8111EA
:104260003ACF0CC0243031050CF039CF9F7009F4DF
:1042700032CFF7019581907F09F02DCF8C2D61967B
:104280000FB6F894DEBF0FBECDBFDF91CF911F9167
:104290000F91FF90EF90DF90CF90BF9008951F9304
:1042A000CF93DF93CDB7DEB72C970FB6F894DEBF70
:1042B0000FBECDBF4F83588769877A878B879C87CE
:1042C000CE0107960E946E1F882369F08F81988522
:1042D0002A853B85232BF1F19F3F09F063C08F3F77
:1042E00009F060C037C086E0FE013796DE01119606
:1042F00001900D928A95E1F76F817885EA85FB85BB
:10430000309741F17F3F11F46F3F21F120912B0352
:1043100030E0C90101968770992740912A0350E047
:104320008417950709F447C069837A83FD83EC837A
:1043300096E0929FD001939FB00D1124A45DBC4FD5
:10434000FE01319601900D929A95E1F780932B032F
:104350000E94E41E16E080912A0390912B03891796
:10436000C1F1189FC0011124845D9C4F0E946E1FF3
:10437000882379F1E0912A031E9FF0011124E45D66
:10438000FC4F4081518162817381848195810E94BB
:10439000D41E80912A0390E001968770992780931C
:1043A0002A03D9CF4F81588569857A858B859C856D
:1043B0000E94D41ECFCF0E946A1E10922B0310922F
:1043C0002A03ECE5F3E086E0DF011D928A95E9F728
:1043D000C1CF2C960FB6F894DEBF0FBECDBFDF91D4
:1043E000CF911F910895DF92EF92FF920F931F9349
:1043F000CF93DF93FC01892B09F48AC0E12CF12CC7
:10440000DD24D394EF0121968491853709F461C0AE
:1044100058F4843708F04EC0843008F06AC0813008
:10442000D1F0823071F174C0883709F45DC050F466
:10443000863709F455C0873709F06AC08E2D0E946F
:10444000DF2454C09CE7980F903708F061C08F7745
:104450000E94E81A50C08F010E5F1F4FFE01849129
:1044600090E2980F983050F48770FD2D01C0FF0F37
:104470008A95EAF78F2F0E94E52414C00E947D1AC6
:1044800013C08F010E5F1F4FFE01C49180E28C0F9D
:10449000883060F4C7708D2D01C0880FCA95EAF787
:1044A0000E94EB240E941625E80125C08C2F0E9453
:1044B000E81AFACF9F012E5F3F4FFE01C491CC2333
:1044C00069F08FE99FE00197F1F700C00000C1504B
:1044D000F6CF9F012E5F3F4FFE01F490E9010BC024
:1044E0000E94CF24E82E07C00E94E2240E941625D5
:1044F00002C00E947D1A8F2D882341F0EFE9FFE072
:104500003197F1F700C000008150F6CFFE017ACF5D
:10451000DF91CF911F910F91FF90EF90DF90089561
:104520006093E2037093E3038093E4039093E503C5
:104530000C94972508956093E6037093E7038093A6
:10454000E8039093E9030C9496250F931F93009131
:10455000E6031091E7032091E8033091E903602B13
:10456000712B822B932B6093E6037093E703809368
:10457000E8039093E9031F910F910C9496250F93F4
:104580001F930091E6031091E7032091E803309117
:10459000E90360237123822393236093E6037093DE
:1045A000E7038093E8039093E9031F910F910C9424
:1045B00096250F931F930091E6031091E703209136
:1045C000E8033091E90360277127822793276093DE
:1045D000E6037093E7038093E8039093E9031F9148
:1045E0000F910C94962560E070E0CB010C94902222
:1045F0000F931F9341E050E060E070E08A019B015F
:1046000004C0000F111F221F331F8A95D2F7C90162
:10461000B8011F910F910C9490220F931F9341E0CA
:1046200050E060E070E004C0440F551F661F771F24
:104630008A95D2F78091E2039091E303A091E4037D
:10464000B091E5038A019B01082B192B2A2B3B2BE8
:10465000C901B8011F910F910C9490220F931F93E1
:1046600041E050E060E070E004C0440F551F661F59
:10467000771F8A95D2F740955095609570958091F7
:10468000E2039091E303A091E403B091E5038A0172
:104690009B01082319232A233B23C901B8011F9139
:1046A0000F910C9490220F931F9341E050E060E033
:1046B00070E004C0440F551F661F771F8A95D2F71C
:1046C0008091E2039091E303A091E403B091E503AC
:1046D0008A019B01082719272A273B27C901B8010E
:1046E0001F910F910C9490220F931F930091E2035E
:1046F0001091E3032091E4033091E503602B712BCB
:10470000822B932B1F910F910C9490220F931F9348
:104710000091E2031091E3032091E4033091E5035B
:1047200060237123822393231F910F910C94902275
:104730000F931F930091E2031091E3032091E40390
:104740003091E50360277127822793271F910F91EE
:104750000C94902208958F929F92AF92BF92DF9215
:10476000EF92FF920F931F93CF93DF9300D000D06F
:104770001F92CDB7DEB76B837C838D838A018C81DA
:104780009D81892B21F01F3F29F44F3F19F480E0D0
:1047900090E04CC08B818823C9F18090E603909013
:1047A000E703A090E803B090E9038091E2039091C1
:1047B000E303A091E403B091E503882A992AAA2A89
:1047C000BB2A8FE1E82EF12CD501C4010E2C04C0C8
:1047D000B695A795979587950A94D2F780FF07C05D
:1047E000DE2CB8018E2D0E94D026019729F481E09D
:1047F000E81AF10848F7D12C88E0189FF00111243D
:10480000E00FF11DEE59FC4FD08209C088E0189FDF
:10481000F0011124E00FF11DEE59FC4FD080098307
:104820001A8369817A818D2D0E94D0260F900F9076
:104830000F900F900F90DF91CF911F910F91FF90EC
:10484000EF90DF90BF90AF909F908F9008959091E0
:104850002001992321F090912101911109C020910B
:10486000220130912301F90132969FEF40E030C0E0
:10487000982F9695969596959F31A0F4E0912201F8
:10488000F0912301E90FF11D877021E030E0A901CB
:1048900002C0440F551F8A95E2F7CA019181892B06
:1048A0008183089590910F0490FF23C01F928F93EE
:1048B0008AE397E09F938F930E94FB070F900F90DE
:1048C0000F900F9008959F3F39F04F5F4E3141F0A8
:1048D00051915813F8CF0DC05111F7CF942FF5CF48
:1048E0009F3F39F0F901E90FF11D97FDFA95828399
:1048F0000895089590912001992321F0909121012C
:10490000911109C02091220130912301F9013296C1
:10491000205E3F4F30C0982F9695969596959F3183
:10492000A8F4E0912201F0912301E90FF11D8770B5
:1049300021E030E0A90102C0440F551F8A95E2F73B
:10494000CA018095918189238183089590910F04F4
:1049500090FF16C01F928F938CE197E09F938F93E7
:104960000E94FB070F900F900F900F9008953196C3
:10497000E217F30729F090819813F9CF1082F7CF4F
:10498000089581E090E0E0912201F0912301E80F89
:10499000F91F1082019680329105A9F70895809140
:1049A0000E04089590910E04892B80930E040895AF
:1049B000809590910E04892380930E04089580932E
:1049C0000E04089510920E04089590910D04892B01
:1049D00080930D040895809590910D048923809310
:1049E0000D04089510920D0408958093EC030E9425
:1049F0000D269093EB038093EA0308951092EC0345
:104A00001092EB031092EA03089580912201909195
:104A10002301FC0131969C01205E3F4F80E0919183
:104A200091118F5FE217F307D1F70895E09122010A
:104A3000F091230180910E048083E0912201F09196
:104A40002301908180910D04892B80838091EC0358
:104A50008823D9F10E940D262091EA033091EB03BF
:104A60008217930748F00E940D262091EA033091A7
:104A7000EB03821B930B0AC00E940D262091EA03D0
:104A80003091EB0320953095820F931F8C3291402B
:104A900070F080910F0480FF08C088E597E09F9335
:104AA0008F930E94FB070F900F900E94FE24E091CD
:104AB0002201F091230190818091EC03892B808366
:104AC0000E94052581110E94FE248091220190916F
:104AD00023010C94AF189093A1018093A001089535
:104AE0008295982F9C7C392F36953695282F2373E5
:104AF00044E0249FC0011124932F982B292F2A7A58
:104B00002695892F8575880F822B08950895CF9358
:104B1000DF9300D000D01F92CDB7DEB70F900F907B
:104B20000F900F900F90DF91CF9108950895089501
:104B30000C94061A80912504843021F110921004FF
:104B400020E488E190E00FB6F894A8958093600087
:104B50000FBE2093600083B7817F846083BF83B7DB
:104B6000816083BF7894889583B78E7F83BF0FB6AB
:104B7000F894A895809160008861809360001092FD
:104B800060000FBE0895CF930E942B090E94420837
:104B90000E942D09C0E08C2F0E942209811104C0BF
:104BA000CF5FC031C1F701C081E0CF9108950E946D
:104BB000081A0C946A1E1F920F920FB60F921124BE
:104BC0008F939F93AF93BF9380911004811113C073
:104BD0008091110490911204A0911304B0911404D7
:104BE0004196A11DB11D8093110490931204A093CE
:104BF0001304B0931404BF91AF919F918F910F90C4
:104C00000FBE0F901F90189582E084BD93E095BD74
:104C10009AEF97BD80936E0008952FB7F894809116
:104C2000110490911204A0911304B09114042FBFA9
:104C300008952FB7F8946091110470911204809137
:104C40001304909114042FBF0895CF92DF92EF9236
:104C5000FF920F931F932FB7F89440911104509136
:104C6000120460911304709114042FBF6A017B0138
:104C7000EE24FF248C0120E030E0C016D106E206CD
:104C8000F30610F4415051099A01281B390BC90150
:104C90001F910F91FF90EF90DF90CF900895CF92EA
:104CA000DF92EF92FF920F931F932FB7F894C0906B
:104CB0001104D0901204E0901304F09014042FBF5C
:104CC00097018601061B170B280B390BC616D70652
:104CD000E806F90618F0C901B80106C0C901B80113
:104CE00061507109810991091F910F91FF90EF9017
:104CF000DF90CF9008951F920F920FB60F9211245C
:104D00008F939F93AF93BF9380911104909112045E
:104D1000A0911304B09114040196A11DB11D8093BC
:104D2000110490931204A0931304B0931404BF9140
:104D3000AF919F918F910F900FBE0F901F9018957C
:104D40000E94B715F8942FEF87EA91E62150804032
:104D50009040E1F700C0000087E090EBDC01809319
:104D60002E0490932F04A0933004B09331049CE060
:104D700088E10FB6F894A895809360000FBE9093D9
:104D80006000FFCF28E0929FF0011124E80FF11D91
:104D9000EE58FE4F9491892F8F7092959F700895D1
:104DA000CF93C82FCB010E94C226282F30E080E18C
:104DB000989FA0011124422B532B4038510519F420
:104DC00080E090E015C09770E92FF0E088E0C89F80
:104DD000E00DF11D112484E0EE0FFF1F8A95E1F72D
:104DE000E20FF31FEE0FFF1FE050F84985919491F9
:104DF000CF91089580E090E0089508958091170480
:104E000080FF0BC06091270185E0689FB0011124ED
:104E100075956795759567952BC081FF09C0609161
:104E2000270185E0689FB00111247595679520C022
:104E300082FF07C06091270185E0689FB0011124BF
:104E400017C0909118049923D1F06091260196170C
:104E500088F72091270185E0289F90011124929FD7
:104E6000A001939F500D112470E0CA010E94E62E0C
:104E70006038710540F46115710539F002C065E0D4
:104E800070E0862F08958FE7089581E0089580915E
:104E9000170480FF08C06091250170E07595679543
:104EA0007595679521C081FF06C06091250170E06E
:104EB0007595679519C082FF04C06091250170E067
:104EC00010C0909118049923C1F0609124019617A5
:104ED000A0F780912501899FC001112470E00E94F4
:104EE000E62E6038710528F46115710521F0862FD2
:104EF00008958FE7089581E0089561E070E0F4CFB0
:104F0000803F21F40E94FE26819504C0813F29F450
:104F10000E94FE2680931B040895823F21F40E9484
:104F2000FE26819504C0833F29F40E94FE268093CB
:104F30001A040895893F19F40E94472705C08A3F43
:104F400031F40E944727819580931C0408958B3F7C
:104F500021F40E944727819504C08C3F29F40E94C8
:104F6000472780931D040895843F21F480911904FC
:104F7000816017C0853F21F480911904826011C0BF
:104F8000863F21F48091190484600BC0873F21F48F
:104F900080911904886005C0883F31F4809119041C
:104FA00080618093190408958D3F21F48091170446
:104FB00081600BC08E3F21F480911704826005C090
:104FC0008F3F29F48091170484608093170408951B
:104FD000803F39F480911B0487FF6CC010921B0442
:104FE00069C0813F29F480911B041816BCF362C08C
:104FF00090911A04823F29F497FF5CC010921A0422
:1050000059C0833F19F41916CCF354C0893F41F4B9
:1050100080911C0418160CF04DC010921C044AC05C
:105020008A3F29F480911C0487FF44C0F6CF8B3F50
:1050300039F480911D0487FF3DC010921D043AC0D1
:105040008C3F29F480911D041816BCF333C0843FB3
:1050500021F4809119048E7F17C0853F21F480913F
:1050600019048D7F11C0863F21F4809119048B7F34
:105070000BC0873F21F480911904877F05C0883FCA
:1050800031F4809119048F7E8093190413C08D3FF1
:1050900021F4809117048E7F0BC08E3F21F4809104
:1050A00017048D7F05C08F3F29F4809117048B7FF3
:1050B0008093170480911A0481110EC080911B0403
:1050C00081110AC080911C04811106C080911D04C9
:1050D000811102C010921804089580910F0483FF7B
:1050E0007EC081E997E00E946207809119041F92B7
:1050F0008F938CE897E09F938F930E94FB078AE839
:1051000097E00E94620780911A04282F082E000C55
:10511000330B3F938F9387E897E09F938F930E9481
:10512000FB0785E897E00E94620780911B04282F07
:10513000082E000C330B3F938F9382E897E09F93E8
:105140008F930E94FB0780E897E00E94620780919E
:105150001C04282F082E000C330B3F938F938DE7F0
:1051600097E09F938F930E94FB078BE797E00E9445
:10517000620780911D04282F082E000C330B3F93EB
:105180008F9388E797E09F938F930E94FB0785E7B3
:1051900097E00E946207809118041F928F9382E724
:1051A00097E09F938F930E94FB0780E797E00E9410
:1051B0006207809117041F928F938DE697E09F936B
:1051C0008F930E94FB078AE697E00E9462078DB7E3
:1051D0009EB74C960FB6F8949EBF0FBE8DBF89E167
:1051E00094E00E94F8180E940D2690931604809374
:1051F000150408951F93CF93DF9380911504909128
:1052000016040E942526AC0190911804992321F0E0
:105210002091280130E006C0209129018AE0289FD2
:10522000900111244217530708F485C080911A0495
:10523000C0911B04D0911C0410911D04811107C062
:10524000C11175C0D11173C0111171C074C09F3FDD
:1052500019F09F5F90931804181624F40E94FE26FC
:1052600080931A0480911A0487FF05C00E94FE26CD
:10527000819580931A041C1624F40E94FE268093C4
:105280001B0480911B0487FF05C00E94FE268195A8
:1052900080931B0460911A04662331F1C0911B04B2
:1052A000CC2311F1062E000C770B880B990B0E9472
:1052B000CD2D23E333E343E35FE30E94312E0E94CD
:1052C000952D60931A046C2FCC0F770B880B990BDC
:1052D0000E94CD2D23E333E343E35FE30E94312EAD
:1052E0000E94952D60931B041D1624F40E944727ED
:1052F00080931C0480911C0487FF05C00E944727EF
:10530000819580931C04111624F40E9447278093F2
:105310001D0480911D0487FF05C00E9447278195C9
:1053200080931D04DF91CF911F910C946D289F3FB6
:1053300009F08FCF97CFDF91CF911F910895E9E1C9
:10534000F4E085E0DF011D928A95E9F710921804D8
:1053500010921704089584EB99E00E9462071F924F
:1053600081E08F931F9285E08F9386E699E09F936B
:105370008F930E94FB070F900F900F900F900F904C
:105380000F9008958330E9F128F4813061F0823084
:1053900009F10895853009F462C008F449C08630E7
:1053A00009F474C0089580912901262F30E0280F58
:1053B000311D2F3F310524F4680F6093290103C08C
:1053C0008FEF80932901809129011F928F938FE99C
:1053D00098E072C080912801262F30E0280F311DFF
:1053E0002F3F310524F4680F6093280103C08FEF2D
:1053F00080932801809128011F928F938DE898E077
:105400005BC080912701262F30E0280F311D2F3FF0
:10541000310524F4680F6093270103C08FEF809358
:105420002701809127011F928F938AE798E044C05B
:1054300080912601262F30E0280F311D2F3F3105A6
:1054400024F4680F6093260103C08FEF8093260138
:10545000809126011F928F9385E698E02DC0809160
:105460002501262F30E0280F311D2F3F310524F470
:10547000680F6093250103C08FEF80932501809111
:1054800025011F928F938CE498E016C0809124012F
:10549000262F30E0280F311D2F3F310524F4680FEF
:1054A0006093240103C08FEF809324018091240135
:1054B0001F928F9381E398E09F938F930E94FB0745
:1054C0000F900F900F900F900895833081F128F482
:1054D000813059F08230D1F00895853009F449C007
:1054E000B8F1863009F456C00895809129016817F3
:1054F00020F4861B8093290102C01092290180911B
:1055000029011F928F9382E298E054C08091280174
:10551000681720F4861B8093280102C0109228018E
:10552000809128011F928F9380E198E043C0809181
:105530002701681720F4861B8093270102C0109270
:105540002701809127011F928F938DEF97E032C042
:1055500080912601681720F4861B8093260102C0E3
:1055600010922601809126011F928F9388EE97E07A
:1055700021C080912501681720F4861B80932501A6
:1055800002C010922501809125011F928F938FEC0C
:1055900097E010C080912401681720F4861B809347
:1055A000240102C010922401809124011F928F9344
:1055B00084EB97E09F938F930E94FB070F900F90CF
:1055C0000F900F900895CF93C82F1F928F9389EB60
:1055D0009AE09F938F930E94FB0781E090E0A0E008
:1055E000B0E0BC01CD0104C0660F771F881F991F72
:1055F000CA95D2F70E949B220F900F900F900F90A8
:10560000CF910C946A1ECF938732A8F58E3108F0A3
:105610002BC1803109F49FC0F8F4873009F464C0CD
:10562000A8F4863009F024C180910F04817F8E7F19
:1056300080930F048EEB9AE00E94620788EA9DE057
:105640000E94620781E080931F044CC08B30F1F10F
:105650008E3009F46CC00CC1863109F4B0C020F45E
:10566000813109F4EDC004C1893109F491C08B3155
:1056700009F449C0FDC0883349F150F4893209F476
:10568000F1C0853309F4EEC0873209F0F1C0EAC0F9
:10569000833409F4E7C028F48A3308F4E9C0895355
:1056A000E4C0883409F0E4C00E946A1E87E99DE0E6
:1056B0000E9462072FEF83ED90E3215080409040DD
:1056C000E1F700C000000E94A0260CC085EE9AE021
:1056D0005CC08EE79DE00E94620780910F048160AC
:1056E00080930F04C1E0C9C080910F04C82FC1701E
:1056F00080FFEFCF8AE89DE00E94620780910F044F
:10570000817F8E7F3DC090910F0491FBCC27C0F923
:1057100081E0C827892FC0FB81F980930F04CC2337
:1057200019F081E79DE027C083E69DE02EC09091AF
:105730000F0492FBCC27C0F981E0C827892FC0FB5A
:1057400082F980930F04CC2319F084E59DE013C007
:1057500084E49DE01AC090910F0493FBCC27C0F91C
:1057600081E0C827892FC0FB83F980930F04CC23E5
:1057700051F088E39DE00E94620780910F048160F0
:1057800080930F047AC08BE29DE00E946207AACF4B
:105790008CE19DE00E9462078FEE9CE00E94620710
:1057A00088EB9CE00E9462078BE89CE00E94620705
:1057B00081E49CE00E94620783E19CE0E6CF85E003
:1057C0009CE00E9462070E94A3181F928F938BEEA9
:1057D0009BE09F938F930E94FB07809120011F9273
:1057E0008F9384ED9BE09F938F930E94FB078091A2
:1057F00012031F928F9381EC9BE09F938F930E94E3
:10580000FB07809121011F928F938EEA9BE09F936B
:105810008F930E94FB070E9419269F938F937F937B
:105820006F9387E99BE09F938F930E94FB078DB74F
:105830009EB746960FB6F8949EBF0FBE8DBF52CF4F
:105840000E946A1EC091210181E0C827C0932101F6
:10585000CC2329F08DE89BE00E9462070EC082E80D
:105860009BE093CF80E001C08D510E94E32A3ACFA4
:1058700080E89BE00E946207C0E08C2FCF910895E2
:10588000CF93C82F80911F04813071F020F08230B7
:1058900009F44BC042C1E0912201F09123018081C3
:1058A000823209F03CC107C0E0912201F09123014E
:1058B0008081823261F48C2F0E946D0C811104C0B2
:1058C0008C2F0E94032B2FC081E090E02CC08C2FE6
:1058D0000E94A10E811126C0C431E1F070F4CB30DA
:1058E00081F0C031D1F40E94AB2981EB9AE00E9493
:1058F000620782E080931F0415C0C93259F0C83393
:1059000061F48EEB9AE00E94620785EB9AE00E94B8
:10591000620708C010921F0404C18FEA9AE00E9437
:105920006207FFC081E08170FEC0C43228F5CE312D
:1059300008F0C1C0CB30A1F1D0F4C73009F0D3C01A
:105940008EE18093290182E3809328018AE080938D
:10595000270184E18093260188E08093250188E275
:105960008093240185E599E00E946207BFC0C3319E
:1059700049F1C431C1F0B7C0CB3409F4A9C028F44F
:10598000C93289F0C83361F0AEC0C13509F49EC098
:10599000C23509F499C0CE3409F0A5C06AE09EC0B2
:1059A0000E94AB29A3C080911E04882319F0109295
:1059B0001E049CC082E699E00E94620781E0809309
:1059C0001F04B1C08CE399E00E9462078AE299E06B
:1059D0000E946207809129011F928F9387E299E0CC
:1059E0009F938F930E94FB0785E299E00E946207D4
:1059F00083E199E00E946207809128011F928F93B2
:105A000080E199E09F938F930E94FB078EE099E0DD
:105A10000E9462078FEF98E00E9462078091270141
:105A20001F928F938CEF98E09F938F930E94FB07B8
:105A30008AEF98E00E94620789EE98E00E94620770
:105A4000809126011F928F9386EE98E09F938F930B
:105A50000E94FB0784EE98E00E9462078FEC98E0BA
:105A60000E946207809125011F928F938CEC98E031
:105A70009F938F930E94FB078AEC98E00E94620735
:105A800083EB98E00E946207809124011F928F931C
:105A900080EB98E09F938F930E94FB078EEA98E03B
:105AA0000E9462078DB79EB748960FB6F8949EBFC6
:105AB0000FBE8DBF1BC0CE51EC2FF0E0EA56FE4F5B
:105AC000808180931E0412C061E003C061E006C0C3
:105AD0006AE080911E040E94C22908C080911E04C1
:105AE0000E94652A03C083E599E013C080911E04DB
:105AF000882369F01F928F938DE499E09F938F9391
:105B00000E94FB070F900F900F900F9004C08AE443
:105B100099E00E94620781E006C010921F0480E0B5
:105B200002C080E000CFCF9108950E949C2D689420
:105B3000B1110C942B2E08950E94102E88F09F57BF
:105B400098F0B92F9927B751B0F0E1F0660F771FA1
:105B5000881F991F1AF0BA95C9F714C0B13091F097
:105B60000E942A2EB1E008950C942A2E672F782FD8
:105B70008827B85F39F0B93FCCF38695779567955C
:105B8000B395D9F73EF490958095709561957F4FC8
:105B90008F4F9F4F0895E89409C097FB3EF490956E
:105BA0008095709561957F4F8F4F9F4F9923A9F0F6
:105BB000F92F96E9BB279395F69587957795679585
:105BC000B795F111F8CFFAF4BB0F11F460FF1BC0C9
:105BD0006F5F7F4F8F4F9F4F16C0882311F096E95C
:105BE00011C0772321F09EE8872F762F05C066230A
:105BF00071F096E8862F70E060E02AF09A95660FC3
:105C0000771F881FDAF7880F9695879597F908957B
:105C100057FD9058440F551F59F05F3F71F047955D
:105C2000880F97FB991F61F09F3F79F08795089542
:105C3000121613061406551FF2CF4695F1DF08C061
:105C4000161617061806991FF1CF8695710561057E
:105C500008940895E894BB2766277727CB0197F926
:105C600008950E94442E0C94B52E0E94A72E38F061
:105C70000E94AE2E20F0952311F00C949E2E0C94D1
:105C8000A42E11240C942B2E0E94082E70F3959FA5
:105C9000C1F3950F50E0551F629FF001729FBB2723
:105CA000F00DB11D639FAA27F00DB11DAA1F649FBF
:105CB0006627B00DA11D661F829F2227B00DA11D72
:105CC000621F739FB00DA11D621F839FA00D611DF8
:105CD000221F749F3327A00D611D231F849F600D19
:105CE000211D822F762F6A2F11249F5750409AF042
:105CF000F1F088234AF0EE0FFF1FBB1F661F771FCE
:105D0000881F91505040A9F79E3F510580F00C9498
:105D10009E2E0C942B2E5F3FE4F3983ED4F3869591
:105D200077956795B795F795E7959F5FC1F7FE2B38
:105D3000880F911D9695879597F9089597F99F6714
:105D400080E870E060E008959FEF80EC0895002403
:105D50000A941616170618060906089500240A94D0
:105D600012161306140605060895092E0394000C56
:105D700011F4882352F0BB0F40F4BF2B11F460FFE5
:105D800004C06F5F7F4F8F4F9F4F0895991B79E03D
:105D900004C0991F961708F0961B881F7A95C9F7BB
:105DA00080950895AA1BBB1B51E107C0AA1FBB1F0A
:105DB000A617B70710F0A61BB70B881F991F5A9597
:105DC000A9F780959095BC01CD01089597FB072E0A
:105DD00016F4009407D077FD09D00E94D22E07FC5C
:105DE00005D03EF4909581959F4F089570956195EB
:105DF0007F4F0895A1E21A2EAA1BBB1BFD010DC007
:105E0000AA1FBB1FEE1FFF1FA217B307E407F5076A
:105E100020F0A21BB30BE40BF50B661F771F881F46
:105E2000991F1A9469F760957095809590959B01DC
:105E3000AC01BD01CF010895EE0FFF1F0590F49155
:085E4000E02D0994F894FFCF56
:105E4800B709BA09BB09BC09BD09B309370A1D0A54
:105E5800B609BE090A01331124120112CD11991194
:105E68000101ED032808140A321E524E2D34320067
:105E78004C554641004F4646004F4E00434F4E4E4C
:105E880000506F776572656400556E617474616364
:105E98006865640044656661756C74004164647289
:105EA800657373656400436F6E66696775726564D0
:105EB800003F0053757370656E64656400404D362D
:105EC8002239840637060106DF05A60519053205BD
:105ED8004B0564058405010203040506070809004B
:1068000088000000000000000400050006000700EA
:10681000080009000A000B000C000D000E000F001C
:1068200010001100120013001400150016001700CC
:10683000180019001A001B001C001D001E001F007C
:10684000200021002200230024002500260027002C
:10685000280035002A002B002C002D002E002F00D0
:1068600030000000320033003400290036003700C9
:106870003800E00000000000000000000000000000
:106880000000000000000000000000000000000008
:1068900000000000000000000000000000004F00A9
:1068A00050005100520000000000000000000000F5
:1068B00000000000000000000000000000000000D8
:1068C00000000000000000000000000000000000C8
:1068D00000000000000000000000000000000000B8
:1068E0000000000000000000890087008A008B0083
:1068F000F1A1E100E200E300F1A1E500E600000003
:106900000100000000000000EA4401000100E24430
:106910000100010001005500460054004A004B00F0
:10692000560057004700480001000100E9440100FB
:106930000100010001000100010001003A003B00DC
:106940003C003D003E003F0040004100420043004B
:10695000580001004C00390001004400450052007D
:1069600001000000010050004F0081404D004E002A
:1069700051000100000000000000000000000000C5
:106980000000000000000000000000000000000007
:1069900000000000000000000000000000004D00AA
:1069A0004A004E004B000000000000000000000004
:1069B00000000000000000000000000000000000D7
:1069C00000000000000000000000000000000000C7
:1069D00000000000000000000000000000000000B7
:1069E000000000000000000049000100010001005B
:1069F0000100010001000100010001000100000090
:00000001FF
